:0200000480007A
:100000006F000005732F2034930F80006308FF03F7
:10001000930F90006304FF03930FB0006300FF038E
:10002000130F000063040F0067000F00732F2034CC
:1000300063540F006F00400093E19153171F0000BD
:1000400023223FFC171F000023200FFC6FF01FFF2F
:100050009300000013010000930100001302000050
:100060009302000013030000930300001304000038
:100070009304000013050000930500001306000020
:100080009306000013070000930700001308000008
:10009000930800001309000093090000130A0000F0
:1000A000930A0000130B0000930B0000130C0000D8
:1000B000930C0000130D0000930D0000130E0000C0
:1000C000930E0000130F0000930F0000732540F102
:1000D0006310050097020000938202017390523072
:1000E000735044749702000093820201739052305F
:1000F00073500018970200009382420273905230AE
:100100009B021000939252039382F2FF7390023B82
:100110009302F0017390023A73504030970200004E
:1001200093824201739052307350203073503030BC
:100130009301000097020000938202ED7390523009
:10014000130510001315F501635C05000F00F00F97
:10015000930110009308D005130500007300000000
:1001600093020000638A020073905210B7B200003D
:100170009B829210739022307350003097020000DF
:100180009382420173901234732540F17300203042
:10019000930120009300100013010000339720000A
:1001A00093031000631C775E9301300093001000EE
:1001B0001301100033972000930320006310775E33
:1001C000930140009300100013017000339720004A
:1001D000930300086314775C9301500093001000B0
:1001E0001301E00033972000B74300006318775AEB
:1001F00093016000930010001301F0013397200079
:100200009B0310009393F301631A775893017000D6
:100210009300F0FF13010000339720009303F0FFD9
:10022000631E7756930180009300F0FF13011000C6
:10023000339720009303E0FF6312775693019000F9
:100240009300F0FF1301700033972000930300F830
:10025000631677549301A0009300F0FF1301E000B0
:1002600033972000B7C3FFFF631A77529301B000A2
:100270009300F0FF1301F00133972000B7030080D3
:10028000631E77509301C000B72021219B8010127C
:100290001301000033972000B72321219B83131201
:1002A000631E774E9301D000B72021219B8010124E
:1002B0001301100033972000B74342429B8323244D
:1002C000631E774C9301E000B72021219B80101220
:1002D0001301700033972000B71309019B8393909B
:1002E0009393C30093830308631A774A9301F00042
:1002F000B72021219B8010121301E00033972000CA
:10030000B72321219B8313129393E300631877484B
:1003100093010001B72021219B8010121301F001ED
:1003200033972000B72321219B8313129393F3016A
:100330006316774693011001B72021219B8010128C
:10034000130100FC33972000B72321219B83131254
:100350006316774493012001B72021219B8010125E
:10036000130110FC33972000B74342429B832324A0
:100370006316774293013001B72021219B80101230
:10038000130170FC33972000B71309019B839390EE
:100390009393C30093830308631277409301400152
:1003A000B72021219B8010121301E0FC339720001D
:1003B000B72321219B8313129393E3006310773EAD
:1003C00093015001B72021219B8010121301F0FFEF
:1003D000339720009B03F0FF9393F3036310773C64
:1003E00093012003930010001301F00333972000C2
:1003F0009B03F0FF9393F3036312773A9301300367
:100400009300F0FF13017002339720009B03F0FF6D
:10041000939373026314773893014003B72021212B
:100420009B8010121301B00233972000B723010004
:100430009B8313129393B302631277369301600187
:100440009300100013017000B39020009303000884
:100450006396703493017001930010001301E00063
:1004600033912000B7430000631A71329301800179
:1004700093003000B39010009303800163907032BA
:10048000930190011302000093001000130170000B
:100490003397200013030700130212009302200079
:1004A000E31452FE93030008631A732E9301A00114
:1004B00013020000930010001301E00033972000A6
:1004C0001300000013030700130212009302200020
:1004D000E31252FEB74300006312732C9301B00184
:1004E00013020000930010001301F0013397200065
:1004F0001300000013000000130307001302120092
:1005000093022000E31052FE9B0310009393F3012B
:10051000631673289301C0011302000093001000BA
:100520001301700033972000130212009302200081
:10053000E31652FE93030008631277269301D0015D
:1005400013020000930010001301E00013000000EC
:10055000339720001302120093022000E31452FE8E
:10056000B7430000631C77229301E00113020000EF
:10057000930010001301F0011300000013000000AD
:10058000339720001302120093022000E31252FE60
:100590009B0310009393F301631277209301F00102
:1005A00013020000930010001300000013017000FC
:1005B000339720001302120093022000E31452FE2E
:1005C00093030008631C771C9301000213020000D0
:1005D00093001000130000001301E000130000005E
:1005E000339720001302120093022000E31252FE00
:1005F000B74300006314771A93011002130200003E
:100600009300100013000000130000001301F0011C
:10061000339720001302120093022000E31252FECF
:100620009B0310009393F301631A77169301200242
:100630001302000013017000930010003397200094
:100640001302120093022000E31652FE93030008E7
:100650006316771493013002130200001301E000C7
:1006600093001000130000003397200013021200C3
:1006700093022000E31452FEB74300006310771288
:1006800093014002130200001301F00193001000D7
:100690001300000013000000339720001302120023
:1006A00093022000E31252FE9B0310009393F30188
:1006B0006316770E930150021302000013017000BD
:1006C0001300000093001000339720001302120063
:1006D00093022000E31452FE930300086310770C8A
:1006E00093016002130200001301E00013000000F8
:1006F0009300100013000000339720001302120033
:1007000093022000E31252FEB743000063187708FB
:1007100093017002130200001301F00113000000A6
:100720001300000093001000339720001302120002
:1007300093022000E31252FE9B0310009393F301F7
:10074000631E7704930180029300F00033111000C0
:10075000930300006314710493019002930000025C
:100760003391000093030002631A71029301A00207
:10077000B310000093030000639270029301B00273
:1007800093000040371100001B01018033902000CE
:100790009303000063147000631030020F00F00F29
:1007A000638001009391110093E111009308D0053B
:1007B00013850100730000000F00F00F930110007B
:1007C0009308D0051305000073000000731000C0EB
:1007D0000000000000000000000000000000000019
:1007E0000000000000000000000000000000000009
:0C07F000000000000000000000000000FD
:1010000000000000000000000000000000000000E0
:1010100000000000000000000000000000000000D0
:1010200000000000000000000000000000000000C0
:1010300000000000000000000000000000000000B0
:081040000000000000000000A8
:040000058000000077
:00000001FF
